:1000000000308A005B2B0000FF00030E8301A1007B
:100010007F08A0000A08A8008A01A00E0408A20018
:100020007708A3007808A4007908A5007A08A6003C
:100030007B08A700831383128B1E20280B196D28C1
:10004000220884002308F7002408F8002508F90096
:100050002608FA002708FB0028088A00210E8300E2
:10006000FF0E7F0E09000A108A100A11820707345A
:100070000F34003407340F34023407340F3404349F
:1000800007340F34083407340F34103407340F3476
:10009000203407340F34053407340F34093407345F
:1000A0000F3411340A108A100A11820709340234FD
:1000B0005108F8015002031860285008F7006C2816
:1000C000F7010830D200D00DF70D51087702031860
:1000D000F700F80DD20B63287A28AD0B732819307E
:1000E000AD00AE0A29147530CF002D08D0000330C2
:1000F000D1005828F708031D7F287430CF0001086D
:10010000CE004F08CE074E0881000B118A1120281F
:100110008501860118306500FF3066008316811363
:1001200083127A2BF801F901F701FA014A08031D3D
:100130009C2849080319B6281030CB000310C70DBE
:10014000C80DF70DFA0D4A087A02031DA9284908BF
:100150007702031CB2284908F702031CFA034A0875
:10016000FA020314F80DF90DCB0B9E2800000034A1
:100170001030F700FA01CD01CA0CC90C031CC628C7
:100180004B08FA070318CD0A4C08CD07CD0CFA0C22
:10019000F90CF80CF70BBC2800340330C8002030F1
:1001A000C700CA013308C90092207908C80078083E
:1001B000C7007908CA007808C900CC014608CB00FE
:1001C000B8207908B5007808B4003508FA0034087A
:1001D0000319B503B403C7007A08C800C708031D94
:1001E000F428C808031917294B30F700F70BF62835
:1001F000000000004B30F700F70BFC280000000067
:100200004B30F700F70B0229000000004B30F700DD
:10021000F70B0829000000004B30F700F70B0E2900
:10022000000000000000000000000000E52800348D
:100230000330C8002030C700CA013308C90092202B
:100240007908C8007808C7007908CA007808C9008A
:10025000CC014608CB00B8207908B5007808B40076
:1002600085143508FA0034080319B503B403C70030
:100270007A08C800C708031D4029C80803195F2968
:100280004B30F700F70B4229000000004B30F7001D
:10029000F70B4829000000004B30F700F70B4E2900
:1002A000000000004B30F700F70B5429000000005D
:1002B0004B30F700F70B5A29000000003129851058
:1002C0000034C508031D67290530C600CD20450848
:1002D000013C03187D290310C50C031C762903304B
:1002E000C60018210130C600CD207C290130C6008F
:1002F00018210130C600CD2067290230C600CD206C
:1003000000340530B300051E83290D30C50061217E
:10031000AA012A0883169B00FF309A001C1583123D
:100320000B08F7008B13831655309D00AA309D00F3
:100330009C149C1899291C11770883128B04051AA8
:100340009F290608FF3AAC002A0883169B008312F7
:100350002C0883169A001C1583120B08F7008B13C8
:10036000831655309D00AA309D009C149C18B62918
:100370001C11770883128B042A0883169B009C1398
:100380001C141A088312C200C5006121AA0A2C0F8E
:10039000892963007C2B3C30BD003D30BC000A3015
:1003A000BE007F2B1930AD00AE01AF010130B800A7
:1003B000A91583160108C0390738810074308312EB
:1003C00081008B16C0308B0400343D082E02031CC4
:1003D000F329AE01AF0AB80A380837020318F22928
:1003E0000130B800A9153E082F02031CFC29AF01FB
:1003F000B108031DB1032915003483169B019C131A
:100400001C141A08FF3C0319342A07308312C60053
:10041000CD20AA012A08013C031C152A2A085220D3
:10042000C200C5006121AA0A0A2A0730C600CD20F1
:10043000AA012A0883169B009C131C141A08FF3C6F
:100440000319342A83123C082E020318312A2A0881
:1004500083169B009C131C141A088312C200C5004B
:100460006121AA0A192A8316831200340608AC00F7
:10047000FF30AC062C083F39C10000302C1B013086
:10048000F700F70DF70DFC30F7057708083EB300CD
:100490004108C5006121E521291D502AFD212911AE
:1004A000362A812BF701F801430803104418F70797
:1004B000F70CF80CC418F707F70CF80C4419F707F9
:1004C000F70CF80CC419F707F70CF80C441AF707E7
:1004D000F70CF80CC41AF707F70CF80C441BF707D5
:1004E000F70CF80CC41BF707F70CF80C00340608DF
:1004F000AC00FF30AC062C080739B9000130B90751
:100500002C083839B700B70CB70CB70C1F30B7053B
:100510000130B707370B8D2AB90100302C1B013091
:10052000C2001E30C3004208C400522278081E3E9A
:10053000BD00822B01303D02BC000230C8005830A3
:10054000C700CA013D08C90092207808BE00C20158
:10055000C3012A0883169B009C131C141A08FF3C35
:100560000319F92A8312C3012830C200AA012A08FC
:1005700083169B009C131C141A08FF3C0319E92ADC
:1005800083122A0883169B009C131C141A088312DA
:10059000B200B208031DD02A0830C2070318C30AEC
:1005A0003208013C0318E22A0310B20C031CDD2AB6
:1005B0000630C2070318C30AE12A0230C207031833
:1005C000C30AD02A0230C2070318C30AAA0AB72AEC
:1005D000831614308312B3004308C8004208C700D2
:1005E000CA013308C90092207908C3007808C20004
:1005F0008316831242083C02BB00B1010130BA00ED
:10060000832B0515851D022BD2213008B100390836
:10061000BA00852BB10803191F2BE52100302918DA
:100620000130013C031D1C2B0230A906A9181A2B0E
:1006300005111B2B05152910B108031D0D2B0511E4
:10064000872BE52138083A020319292BBA08031D24
:10065000592B0030A9190130013C031D592BA91158
:1006600005140830B3003B082E020318512B073045
:10067000C600CD20AA012A08023C031C502B3B08CF
:100680002E0203184E2B3908C3000330C400522237
:100690002A0878073320C400C5006121AA0A3B2B31
:1006A000332B1430B300FD213C082E02031C542BC5
:1006B0000510212B882B84011F30830507309F00F4
:1006C0002910A9102911A911AA01AB01AC01AD0192
:1006D000AE01AF01B001B101B201B301B401B50186
:1006E000B601B701B801B901BA01BB01BC01BD0136
:1006F000BE018828051E8129861F812BCB29D22186
:10070000362A772A9A2A851D012BD2210A2B212BE2
:02071000630084
:02420000FF00BD
:02400E0041036C
:00000001FF
